S0180000746F7765725F626F6F746C6F616465722E7372656351
S1130000F885FF1F11040000EB04000071290000B3
S11300107329000075290000772900000000000002
S1130020000000000000000000000000EB040000DD
S1130030EB04000000000000EB0400008308000053
S11300407B3A00007B3A00007B3A00007B3A0000D8
S11300507B3A00007B3A00007B3A00007B3A0000C8
S11300607B3A00007B3A00007B3A00007B3A0000B8
S11300707B3A00007B3A00007B3A00007B3A0000A8
S11300807B3A00007B3A00007B3A00007B3A000098
S11300907B3A00007B3A00007B3A00007B3A000088
S11300A0E72F0000EB2F00008D2B0000912B0000A8
S11300B07B3A00007B3A00007B3A000021350000C7
S11300C07B3A00002D3500007B3A000049350000E2
S11300D07B3A00007B3A00007B3A00007B3A000048
S11300E07B3A00007B3A00007B3A00007B3A000038
S11300F07B3A00007B3A00007B3A00007B3A000028
S11301007B3A00007B3A00007B3A00007B3A000017
S11301107B3A00007B3A00007B3A00007B3A000007
S11301207B3A00007B3A00007B3A00007B3A0000F7
S1130130A30900007B3A00007B3A00007B3A0000F0
S11301407B3A00007B3A00007B3A00007B3A0000D7
S11301507B3A00007B3A00007B3A00007B3A0000C7
S11301607B3A00007B3A00007B3A00007B3A0000B7
S11301707B3A00007B3A00007B3A00007B3A0000A7
S1130400FFFFFFFFFFFFFFFFFFFFFFFFFEFFFFFFF9
S113041072B60E480E49886000220023002400258D
S113042000260027B846B946BA46BB46BC4609482A
S1130430854609488047094880470948804762B68D
S113044000200021074A9047FEE70000000000005A
S113045000ED00E0F885FF1FA5380000B121000081
S1130460EB210000C91A0000000000000000000099
S1130470002A01D101207047F0B41F46034603242B
S11304802340002B09D00424E31A0170013008240E
S1130490E141521E26D05B1EF7D1042A1ADB13D089
S11304A0002F11D00C460D460E46102A02DB72C0F6
S11304B0103AFAE70C2A02DB32C00C3AFAE7082AAF
S11304C002DB12C0083AFAE7042A03DB01600430B5
S11304D0121FF9E7002A05D0017001300824E14118
S11304E0521EF7D1F0BC00207047FEE7790B0000E4
S11304F0000000008B0B000000000000210C000035
S11305006F0D00000F0C0000930C0000430E000060
S113051000000000E10E000000000000C50B000018
S1130520000000009F0B0000930C0000570E000019
S113053000000000C10E0000000000002F0B0000AE
S113054000000000F90B00000000000000000000A3
S113055000000000F50E0000000000001B0F00006A
S113056000000000570F00006F0D000000000000A5
S1130570000000000000000000000000000102462E
S1130580051B0000931B000000000000B51B0000C9
S11305903B1C0000F11D0000211E0000831E000012
S11305A08F1E0000171F00001D2000000000000027
S11305B0BF1C0000AD1D0000011D0000591B000000
S11305C09B1F00000000000000000000000000006D
S11305D00000000000000000553A00005F3A0000EF
S11305E0693A00000000000000000000512A0000E9
S11305F0932A0000EB2A0000000000000000000025
S11306001F2B0000F91000002911000069110000DF
S11306104F1200000000000089120000EF2F0000BC
S11306202F300000D5300000000000000000000062
S113063011310000032700008D250000B5250000BE
S1130640312600006D260000F125000087240000FB
S11306508B2400009D240000DB2400000000000027
S1130660000000000100000000000000F30800008A
S1130670D8060000E8060000F006000002000000B2
S113068000000000330900001C0600002C060000D6
S1130690F006000004000000000000005F090000F4
S11306A0EC050000FC050000F0060000000000005E
S11306B00000000000000000000000000000000036
S11306C000000000A5310000E33100000533000004
S11306D0B93300001482FF1F2D340000B134000030
S11306E0CB340000000000000000000005350000CD
S11306F09135000097350000FF3500009D3600005D
S113070095350000A93600007135000038B504465F
S11307103D4D0020C5E90000C5E90200C5E904001B
S113072028626862394800F0A0F8C5E9060120464D
S1130730BDE834400FF2550100F044B900F053B95C
S113074070B5314D0C46296A072904BF696A88428D
S11307501AD100F093F8C0EB0016D5E90001D5E9F1
S113076002231018B6FBF0F00A2148434FF49661B7
S1130770B0FBF1F0401D0A21B0FBF1F04FF496619B
S113078048432060002070BD012070BD2DE9F8436E
S1130790064600F05AF81C4F0446386AD7E9045953
S11307A08846421CD7E90601651B68EB09094945DF
S11307B002D82CBFA8420122012A3A6206D0042A98
S11307C008D0052A0ED0072A0FD018E0C7E9004840
S11307D07E6214E0D7E90001201A68EB0101C7E941
S11307E000010CE0C7E9024809E0D7E90201201A38
S11307F068EB0101C7E90201304600F0F4F8C7E9EB
S11308000448BDE8F18300000881FF1F803801001F
S11308101E48002101606FF07F421D494A6000229A
S11308208A6007220A601B491B4A0968C900B1FB98
S1130830F2F101B901214160704715480168C90806
S1130840C900016000218160704710490A6813489B
S113085000680B68C0430002000A9A42F6D10021E6
S113086010EB026051EB1221704708494968A1FB63
S11308700001C00840EA4170C90870470548006893
S1130880704702480168491C016070470882FF1FD5
S113089010E000E00081FF1F40420F0018E000E07C
S11308A00901002806D55B4A00F00F00801800F803
S11308B0041C7047584A8154704750F82130120480
S11308C023F4702302F470221A430FE050F821003D
S11308D0C0F30060704706E0120202F4E06242F0E6
S11308E0200203E000BF120202F4E06240F821207B
S11308F0704700B1704710B5484C19B102290DD0AA
S113090003D310BD2064606410BD4FF48070206474
S11309104348016821F48031016010BD0322102195
S11309202046FFF7D8FF2046BDE8104003221121DE
S1130930D1E700B1704710B53A4C11B1022903D088
S113094010BDA060E06010BD072203212046FFF720
S1130950C3FF2046BDE8104007220221BCE700B1D6
S1130960704710B5304C11B1022905D010BD206478
S11309706064A064E06410BD022210212046FFF7E9
S1130980B1FF022211212046FFF7ACFF02221221FF
S11309902046FFF7A7FF2046BDE81040022213219E
S11309A0A0E780B510211D48FFF790FF48B11F480C
S11309B00168080005D0002088471D494FF0FF302A
S11309C0086001BD10B50C4660B901213C20FFF759
S11309D067FF18494FF0805008600A2200F015F8AC
S11309E01248046010BD00B1704780B512494FF041
S11309F08050086000213C20FFF752FF002200F0E5
S1130A0004F80A490020086001BD1021034854E796
S1130A100000000018ED00E000E400E000A0044045
S1130A2054F00F4000C0044000D004401082FF1F67
S1130A30A0A0044004E100E084E100E0DFF8301607
S1130A40C968C9680020086070472DE9F041DFF8E3
S1130A50205682B0E86900248DF801404669002ED2
S1130A6062D0E968C9680A68012A4CD001F1080219
S1130A7074680023091DA04704001FBF42F21270CE
S1130A80844242F2137084424ED1E868C168D1F8BE
S1130A900880B8F1000F47D04E68377837B1132F6C
S1130AA004DA806800EBC700083800E00020086220
S1130AB000281CBF006800281CD02A699269694676
S1130AC005F120009047040016D19DF8000040B1C4
S1130AD04FF4E750791EC840C00758BF42F2117462
S1130AE00AD5EA68D268126A1268414630469047CD
S1130AF0002406E042F210743946204600F040FA21
S1130B0094B901200DE0086A48B14168080003D097
S1130B100DF10100884704460CB1002001E09DF866
S1130B200100E968C96808602046BDE8F68180B51F
S1130B300178002000F024FADFF83405C069416927
S1130B4009698847022000F09BFABFF34F8FDFF852
S1130B502405DFF82425016801F4E06111430160F4
S1130B60BFF34F8F00BFFDE7DFF80405C068C0681E
S1130B7014210C3000F0B6BA10B5044600F0ACFBFA
S1130B80FFE72178BDE81040FAE110B5DFF8E02472
S1130B90126852690446A16860689047F1E710B58D
S1130BA000F04AF8DFF8C804C068C06861680161F1
S1130BB0082101770020217800F0E2F9BDE8104017
S1130BC000F09FBD30B583B0DFF8A444A5680021D0
S1130BD0019100916B4681684068AD6801AAC9B271
S1130BE0C0B2A847E268D2680021116100998A085E
S1130BF0019900F0D9F937BD10B5DFF87424926873
S1130C00D26804466068A168C0B29047B9E710B5DD
S1130C1000F012F800F012F8042101770020B0E788
S1130C2010B500F009F800F009F80321017700205D
S1130C30A168BDE81040CEE1044695E7DFF8300432
S1130C40C068C068A168016161684161704738B5D6
S1130C5000F088F8002141610161007F042804D17B
S1130C6028680069804704B90446E868C068017FC1
S1130C70204600F085F942F21270844208D1E868F7
S1130C80C068007F082804BFBDE8314000F078BD8B
S1130C9031BD2DE9FC4100F065F8016921B900205E
S1130CA02070FFF7D4FF5AE00121217006694769DB
S1130CB0002000900123E869D0F814C0DCF804C0D7
S1130CC06A4601A9E0475FEA000805D0E86941697E
S1130CD0C9688847404603E0009830B942F2127070
S1130CE0FFF7B5FF002020703AE0B04288BF3046DD
S1130CF00090E868C068017F082913D10199C16098
S1130D00009981610198009900F005FD804642F246
S1130D107D7080451CBF42F2747080450BD14FF04A
S1130D20000808E02B68019A00999B6838469847A8
S1130D3080460098C7190098361A06D0B8F1000FFB
S1130D4009D0E8694169C96888474046FFF77FFFD1
S1130D500020207003E0E868C06806614761002055
S1130D60BDE8F681C24D0446E868C06870472DE9C5
S1130D70F047BF4D8AB00446E868C068016921B9EC
S1130D8000202070FFF763FF57E0012121700669FE
S1130D904769C168027F212E2CBF4FF02008B0465E
S1130DA0A9B1424601A800F043FDE869D0F814C097
S1130DB0DCF808C00123424601A9E047A6EB080677
S1130DC006B1B0B3FFF743FF0020207035E0032ADB
S1130DD008EB070907D12B685B6801AA414638462E
S1130DE09847824614E0102A18BF4F46DDD190F888
S1130DF01DA000F063FD39462F69CDF800A04346DD
S1130E00FF6B01AA05F12000B847824600F05CFDA3
S1130E10BAF1000F4F46C8D0E8694569AD680123AF
S1130E20002201A9A8475046FFF711FF00202070B7
S1130E3004E0E868C0680661476100200AB0BDE8C4
S1130E40F08710B58A4B1B68DB680446E268A1682A
S1130E506068984795E62DE9F0410546874C6E6831
S1130E60D5F80880E8688249206000274968103175
S1130E7030B10A68904223BF4968491C8142042763
S1130E80304600F046FD00B904272978384600F0C2
S1130E9077F89FB96660002000F0F2F82068C4F883
S1130EA0088018B180F3088880F309886168404697
S1130EB08847BDE8F041002000F0E2B8BDE8F081C9
S1130EC038B50446606800F024FD08B9042005E044
S1130ED06568012000F0D4F8A068A847217819E0DB
S1130EE0634A10B5044602F120001269D269211D3B
S1130EF0904746E638B55E4D044600F0DFFC00F04E
S1130F0024F86D6B04F10C02A847054600F0DCFCE4
S1130F1021782846BDE8344032E030B583B0044639
S1130F2068460021002206C0514D00F0C7FC00F0C5
S1130F300CF8AD6B6A46A847054600F0C5FCA268EC
S1130F406946284600F04BF837BD05F120002D69AD
S1130F50A3686168704710B5FFF76EFE4448C16826
S1130F60C968A2680A6162684A6110220A77C06887
S1130F70C068E16841770020A168BDE810405BE0EB
S1130F8010B584B0A02201908DF80020002200F05A
S1130F906AF88DF80220029102228DF803200023C2
S1130FA04469A4680C225BE010B588B0A72300F064
S1130FB03AF80020531C8DF8033006E06C4651F8D3
S1130FC0203004EB8004401CA3609042F6D300F070
S1130FD021F800231AE010B584B0A3222FE010B545
S1130FE088B0AF2300F01FF802238DF8033040B916
S1130FF09008801C8DF80300029203A800F028FCDE
S113100001E000200290002300F004F86946A047A4
S113101008B010BD1648C0699DF803104469A4685F
S113102089000A1D70478DF80030019000238DF867
S113103001308DF80230704710B584B0B0228DF8BD
S113104000200190012200F00EF8029100228DF898
S11310500220002302228DF803200C224469A46894
S11310606946A0471FBD0248C0698DF8012070473A
S11310701080FF1F0CED00E00400FA055481FF1FEF
S113108070B50446022C04D0002001F009F8012CAC
S11310900ED00026114D06E04019C16889680A0087
S11310A018BF8847761C1820704341590029F3D192
S11310B074B900F003FCFFF7C0FB01F096F808498F
S11310C000200860012001F0BDF801F07DF962B64E
S11310D0BFF36F8FBFF34F8F70BD00BF6406000076
S11310E008ED00E0002201F0B5B90000C449EFF3B7
S11310F01080486072B6704738B5C24D2B696C6871
S1131100DB6A2246042105F1200098472B69DB6A3B
S11311106A46012105F120009847206800990818C3
S1131120401E6060002032BDF8B5B64F0446786BAF
S11311300D464042164600EA0401621AAA185242B9
S11311401040424207F120003F697F6C6B46B8476C
S113115048B99DF8000008B16C20F2BD324629461A
S1131160204601F092F9F2BD2DE9F04F89B0924684
S113117080460C4603AA00F01CF906005BD1A708C0
S1131180BF00E41B4FF0FF300690079005D02246C5
S113119007EB0A0106A800F04BFBFFF7A7FF07EBDC
S11311A00809984D4FB12E6976693B46524641462F
S11311B005F12000B047060009D144B12E697669D3
S11311C0042306AA494605F12000B0470646DFF885
S11311D030B2DBF8040080F3108866BB9DF80C0085
S11311E058B3FFF783FF87B104A80290414605A8CE
S11311F00190534600F025F83A462E69D6F8288027
S113120005F12000C047060010D17CB104A802906B
S113121006AB05A80190082200F013F849462C6992
S1131220D4F8288005F12000C0470646DBF8040006
S113123080F310880EB1304600E0002009B0BDE80C
S1131240F08FA8680069006DC0B20090704770B557
S1131250044688B00D4600204DF82020401C082884
S1131260FAD375B12026202D98BF2E466A46314602
S11312702046FFF779FF002804BF3419AD1BF0D0D6
S113128000E0002008B070BDF8B504460D46FFF735
S11312902DFF5C4E5C4B37693F692A46214606F1B7
S11312A02000B847564F796881F3108898B9B1681F
S11312B00969096B79B1FFF719FFB0680069036D1B
S11312C021463469646ADBB22A4606F12000A0474D
S11312D0796881F31088F2BDF8B54A4CA1680969B0
S11312E06668326801F1580589692B6800204F420D
S11312F093421ED16968914225D1FFF7F7FE226916
S1131300414992683E4D04F120009047696881F399
S1131310108868B9A1680969096B39B1FFF7E6FE5D
S113132000F03EF8696881F3108808B9012129703A
S1131330F2BD9A4207D217EA030104D01046FFF720
S1131340A3FF0028F4D16968494239404A427168D0
S11313508A42EDD2481C811A1046BDE8F44093E756
S113136070B5154682B000222A700A46254C2669BB
S1131370766C01466B4604F12000B04778B99DF8BD
S1131380001029709DF8001049B11D4D297831B91C
S113139000F006F808B16C2076BD0121297076BDF5
S11313A0A06800692269016D126AC9B204F12000C3
S11313B0104770B50546134882B080680069006B19
S11313C00E46144600B101202070FFF78FFE7042D4
S11313D08008800041426A462846FFF7C1FF084959
S11313E0496810B181F3108876BD81F310889DF8A7
S11313F0000008B100202070002076BD000000002D
S1131400F081FF1F1080FF1F6B66656B4168826867
S11314108A4209D2891A416082660FF26121016011
S1131420012181600020704742F2787070470FF20A
S1131430050113E0416ADFF8D4334A898282CA681D
S1131440921E42604A689A4202D1097A022902DB5A
S113145042F2757070470FF20D0100BF0160002069
S11314607047000010B5044682B0606A4168626843
S1131470A1610168C91E9142A16002D342F2767053
S113148016BD008910B142F2777016BD8DF80000C8
S11314906946DFF87C2302F12000126992699047C3
S11314A09DF8000010B142F2817016BD2046FFF78E
S11314B0ADFF16BD38B5DFF858532B689B6804465A
S11314C0626A216EE06D9847A8B9A1682069491E37
S11314D0884203D328680069804760B900F03AF86D
S11314E000F033F80098616E884200D038E00FF2C3
S11314F08D102060002032BD38B50446C44D00F084
S113150029F82B68626AE06D9B6810219847D8B966
S1131510E06D1030E065206E10382066112828BF79
S1131520BC480FD208B1BC480CE028680069804769
S113153050B900F00AF80098616E884200D00FE0BC
S11315400FF239102060002032BD694604F11C00FE
S113155000F0FEBF616A102204F11C0000F0CCBF51
S113156042F27A7032BD10B5044604F11C0000F05A
S1131570BDFF206E11282CBFA648A748C8E0A44B85
S11315801B68426E016EC06DDB681847F8B50446EF
S1131590B4F85A00C0F30321C0074CBF0825042542
S11315A0E66D042901D00420F2BD00F087F904F1AE
S11315B06002974F3C69646B2B46314607F120006B
S11315C0A047044600F080F9002C14BF20460020F8
S11315D0F2BD70B5044642F27F76E56D284600F010
S11315E098F980B1606E04F11801A8470646012EEF
S11315F003D12046BDE8704008E7022E03D100F075
S113160080F8002070BD304670BD10B500F15C015B
S1131610031D1C684A685A60944202D242F27670F2
S113162010BD0A7AD20708D50A685C69A24204D1BF
S1131630496811B19960002010BD90F85A10C9078B
S11316405CBFBDE81040FFF7E1BE42F27C7010BD04
S1131650B0F85A108A0707D4CA0707D5C1F3032084
S1131660002808BFFFF738BE04207047684A126894
S113167052695C30416800681047000070B5044648
S113168004F15805616A2846102200F0E1F85A2650
S11316900120415D7618401C1028FAD32878F1B255
S11316A0884202D042F2797070BD69780A2942F208
S11316B0127023D8DFE801F01A060A0E24121A1653
S11316C0241C1E002046BDE870409EE72046BDE86D
S11316D0704048E72046BDE8704050E72046BDE82A
S11316E0704076E72046BDE87040B1E7002070BD49
S11316F0042070BD2046BDE8704047E742F27B708D
S113170070BD10B5454C70212046FFF7EBFC4448F2
S11317102060002010BDF8B504460D4600200026C8
S1131720404FAE4217D03869C0F11000A91B09E040
S113173079B13B69325DDA55761C3A69521C3A61DB
S1131740401E491E0028F3D1386100F005F810B995
S1131750E7E742F27D70F2BD3049324A4A62002026
S1131760CA682AB10B69934209D0581C086101E088
S11317708A6E12B9084609680847521E8A6670477D
S1131780F8B5234C20680069804700283DD1234FD9
S113179097F85900042824D107F15C052E683046D7
S11317A000F0B7F8D0B10020FFF76AFC97F85A00B0
S11317B0800711D5686868616168103160B10A6892
S11317C0904222BF4968491C814201D20420F2BDE3
S11317D080F3088880F30988A868B04742F27E70D5
S11317E0F2BD08280FD10220FFF74AFCBFF34F8F48
S11317F00D480E4A016801F4E06111430160BFF332
S11318004F8F00BFFDE742F27B70F2BD53544D5041
S11318101080FF1FF9140000B5140000D082FF1FD0
S11318202F1400004483FF1F0CED00E00400FA05B0
S113183062B38B0708D0521E11F8013B00F8013B3C
S113184000F024808B07F6D1830740F0208000BF8E
S1131850103A07D330B4B1E83810103AA0E8381081
S1131860F9D230BC530724BFB1E80810A0E808102F
S113187044BF51F8043B40F8043BD20724BF31F87D
S1131880022B20F8022B44BF0B7803707047083AF0
S113189007D3B1E80810083A40F8043B40F804CBF9
S11318A0F7D25307E4E700000021016062B67047F5
S11318B072B60A490020086062B6704772B60748DB
S11318C00168491C0160704704480168022900D27C
S11318D0EAE70168491E0160704700000082FF1FAB
S11318E038B504460D460020FFF7CAFB7E487F4A00
S11318F0056044604FF420411160016881F3088859
S113190081F3098840688047BDE832400020FFF732
S1131910B7BB10B582B000281EBF10F1010F744987
S1131920884201D1002016BD6A46022100F0AAFEB9
S1131930002418B90098007A00B10124204616BD8D
S11319402DE9F04F6B4E6C4F85B0B068006968307C
S113195000903D460AE00099097C014205D068697F
S1131960EA68816952682846904718352868002833
S1131970F1D10024A246CDE9024A4FF47A70FEF771
S113198074FF05468B460821002000F0CBFE30B9D9
S11319904FF42040D0F80480D0F8009001E0A04635
S11319A0A14600F02BFDA8BB4046FFF7B2FF88B369
S11319B0B068006990F88600C00703D449464046E1
S11319C0FFF78EFF0098408A4FF6FF71884208BFE8
S11319D041F28830A5FB00230BFB0033CDE9022341
S11319E0FEF733FF04468A46DDE90201002908BFF9
S11319F000280FD0FEF729FFDDE90223001B61EB6D
S1131A000A01994206D301D8904203D3494640467D
S1131A10FFF766FF3D4600E0183528680028E3D04C
S1131A200099097C0142F7D0E9680968284688478B
S1131A300028F1D0002DD7D00AE00099097C01429A
S1131A4018BFBD4203D0F9688968384688471837FB
S1131A5038680028F1D1284605B0BDE8F08F10B5EC
S1131A60FFF726FF00F0AAFC224C2169496804F123
S1131A702000884721692148E06304F12000096CB3
S1131A808847A06800688047002000F0DBFBFEF771
S1131A90BFFE206800688047A06840688047FFF761
S1131AA04FFFE061016919B109680A0018BF88474E
S1131AB0E069416919B109680A0018BF8847E068FC
S1131AC00068BDE81040004738B5FFF7C8FF094C6F
S1131AD0E569E06840688047E868C1680800F8D0B4
S1131AE028468847F5E700006081FF1F08ED00E005
S1131AF0110400001080FF1F640600006480FF1FB3
S1131B007047000008B904207047DFF8B015096871
S1131B10090E01F00F010F290FBF4FF400210FF23E
S1131B20706232F8111089020022026041604FF4A1
S1131B308072022181604FF40061C160DFF880157A
S1131B4091F900309A404261C978816100210161B4
S1131B50016241620020704770B508B9042070BD6D
S1131B60C4690FF20C6165680C222846FFF760FE19
S1131B70DFF850650FF20461681C30601422A56818
S1131B802846FFF755FE681C706002202060002084
S1131B9070BD38B5040001D1042032BDDFF828251A
S1131BA06FF03B401060DFF82405814201D06B20C8
S1131BB032BD38E02DE9F04389B0164680460D4623
S1131BC000F0E3F9049B00F0DCF904001BD1009D54
S1131BD0019F7019461EB6FBF7F007FB106121B197
S1131BE0401C7843461E00E07D19AE4217D32802FC
S1131BF0000ADFF8D41440F010600860DFF8CC0469
S1131C00814502D06B24204656E000F082F9044658
S1131C10D8F81000010018BF8047002CE4D04046DB
S1131C2000F03EFAEFE7204600F020FA00F002F858
S1131C30284632BD0546204632E22DE9F04389B0FC
S1131C4004465FEA02080F461D4608BF042033D04D
S1131C5000F09CF9039B2A463946204600F054FACA
S1131C605FEA000928D1009FDFF85C6402E0039872
S1131C70C7192D1AEDB158F8040B70603902039896
S1131C80090A042808BF41F0C06006D0082805D11D
S1131C9058F8040BB06041F0E0603060204600F07A
S1131CA0E5F981462069010018BF8047B9F1000FAA
S1131CB0DDD0FFF7C0FF484609B0BDE8F08370B53A
S1131CC0040018BF002A01D1042070BDDFF8F80316
S1131CD0DFF8FC63CDB246EA0545056010291568B6
S1131CE0456002D01139032903D2082B04BF51687F
S1131CF08160204600F0BAF9FFF79CFF284670BDCA
S1131D002DE9F04389B05FEA0008914614BFB9F1A8
S1131D10000F04200E461D4647D000F037F9069800
S1131D20401E064208BF05421AD1A919109C002082
S1131D30491E012C05D1002E04BF691E07290AD1B2
S1131D400AE044B9FF2907D9B6F5000F03D3DFF839
S1131D508423914200D3042038BBDFF86C730DE078
S1131D60652022E0796849F8041B0699082904BF14
S1131D70B96849F8041B06998E196D1AADB1300281
S1131D80000A40F0407038602006069940F0FF10C9
S1131D9040F47F40042908BFB86002D0082908BF76
S1131DA0786000F0B6F80028DCD085E7F8B5154671
S1131DB0002818BF002D0C461E4601D10420F2BD98
S1131DC0DFF80473DFF81023E1B242EA014139601D
S1131DD000F04CF958B979682960102C03D0A4F1AB
S1131DE01101032903D2082E04BFB9686960F2BD4A
S1131DF0002818BF002901D104207047DFF8DC0255
S1131E00007800F00302022A08BF002005D000F089
S1131E10C00080280CBF01200220087000207047F9
S1131E2010B50A46002818BF002A01D1042010BDAD
S1131E30DFF8A8321C78002104F00304022C1ED021
S1131E406FF03A41C3F8021054781178240444EA3C
S1131E500161947841EA0421D4782143C3F806103F
S1131E6054791179240444EA01619479D27941EADC
S1131E7004211143C3F80A1000F0F8F8014608469B
S1131E8010BD08B904207047DFF8542280E02DE922
S1131E90F04F89B0924680460C4600F076F8059BD8
S1131EA052462146404600F02FF978BB6A46214647
S1131EB0404600F03EF9009C029E60427142084098
S1131EC04542A54208BF75197F4F03E0AAEB0B0AF0
S1131ED05C447519BAF1000F17D0281BD34682450C
S1131EE088BF83460598BBFBF0F02102090A000471
S1131EF041F0807140EA0920396040F0FF007860C9
S1131F0000F007F80028E1D000E0002009B0BDE8A7
S1131F10F08F4046AAE02DE9F04389B080465FEA9D
S1131F2003090D46164608BF042029D000F02EF8F8
S1131F30079B00F026F818BB009D109C624F05E03B
S1131F4007998A08761A09EB82094D19C6B1280245
S1131F50000A40F000703860200640F0FF1040F4A2
S1131F607F407860D9F80000B860FFF7D2FF0028FE
S1131F70E6D0119901B10D60129909B100220A60ED
S1131F809AE6324629464046BEE099466A46D0E083
S1131F9042EA01414C4A116068E02DE9F041804673
S1131FA01E000D46174608BF042034D0042300F059
S1131FB0ABF880BBD8F814307A195F42C2F1000C38
S1131FC007EA0C0CCCF1000C2F40ACEB0707002106
S1131FD0B7FBF3F7DFF80CC10AE0DCF800E0203CC3
S1131FE06FEA0E0E2EFA04F4E40748BF491C5D198B
S1131FF095420AD2B5FBF3F4202C38BFDCF804E098
S1132000EED3D8F818E07445E7D319B1B94234BF18
S1132010022101213170BDE8F0810000002818BFC1
S1132020002A01D10420704709291DD8DFE801F0F6
S113203005090B0E10121416181AC068106000203F
S113204070474068FAE740684008F7E78068F5E7BA
S11320500068F3E70120F1E74069EFE78069EDE705
S1132060006AEBE7406AE9E76A20704710B51E4C46
S11320707021217000F03CF888B9124909682046A3
S113208088472078810601D5672010BDC10601D597
S1132090682010BDC00701D5692010BD002010BD07
S11320A038B50400200000F023F80500002D03D10A
S11320B00E4804494968884731BD00004C800440FB
S11320C028000240F881FF1F040002406B66656B24
S11320D0FFFF004300048000FFFF004102000240B4
S11320E0FFFF0040180002400000024004F00140DD
S11320F008B904207047C06920B10068022801D1E2
S1132100002070476D20704708B9042070475B1E9B
S1132110194208BF1A4201D06520704703689942EA
S113212021BF4068C0185118884234BF662000207F
S1132130704770B505000E46144601D1042070BDE9
S113214020212046FEF7CEFF2868301A2060E86878
S11321506060A9686868B0FBF1F0A0600420E060EA
S11321600820206160610420A061E061002070BD4E
S11321708021017002780A42FCD070470168F02285
S113218012040A430260BFF36F8FBFF34F8F70478F
S1132190080010001800200030004000600080009B
S11321A0C0000001800100020003000400060000DA
S11321B080B518491848086018491948421A19483E
S11321C088421CBF002AFFF733FB17481749091A36
S11321D018BF00F0BDFA16491648421A04D0BDE8EB
S11321E008401548FFF724BB01BD14484FF0FF31E8
S11321F0016041608160C160016141618161C161CF
S11322000F48016041608160C16001614161816189
S1132210C161704708ED00E00000000008390000CB
S11322200C3A00000080FF1F0881FF1FF483FF1F8A
S1132230DC3A0000DC3A0000F483FF1F80E100E098
S113224080E200E02DE9F041524C534D010020782A
S113225063D12968616051498968096901F168029B
S11322604F49137FDB0708D52868000F4FF0A07291
S1132270401CB2FBF0F0086056E0527F494ED24356
S113228002F00F02521C484BB3FBF2F3B342F9D2F3
S1132290944616461746DFF8148101E00CF1010C50
S11322A0DFF804E1BEFBFCFEC645F7D2DFF8F8E038
S11322B0DFF8FC80BEFBF6FEC64528BF761CF5D2CF
S11322C000E07F1CDFF8E0E0DFF8E880BEFBF7FE0B
S11322D0C645F6D2012A05D1BCF1090F3CBF092E2F
S11322E0092F21D2ACF1010C4FEA0C6C761E521E60
S11322F00CF0706C36054CEA027206F47006324338
S11323007E1E360406F4702632432A600B600121D7
S113231000F00CF80120207006E0012904D100210E
S113232000F004F860682860BDE8F081884230D08D
S1132330012921481BD1417801F0CF0141F020014E
S11323404170017801F0C30141F030010170C1789E
S113235001F09F0141F02001C170017B01F0FC01FB
S113236041F0020101738179C906FCD4704781B937
S1132370017841F0040101708179C906FCD504217A
S1132380017080214170C17801F06001C1700021A9
S113239001737047E881FF1F448004401080FF1FD1
S11323A00081FF1F010E2707006CDC0201879303E5
S11323B081C3C90141787D01004006401D48016880
S11323C041F47851016070471A48016821F478514A
S11323D0016070471848194A016800681268000FC4
S11323E0401CC1F303615043491CB0FBF1F070473A
S11323F0002806BF11480068002070471048016893
S113240041F4807101600F494A6822F040024A6039
S1132410026842F01302026000204FF4FA720B6863
S1132420C3F380131818521EF9D1FA288041C00F43
S11324307047000038800440448004400081FF1F3E
S113244018B0044090F00F407047000062F30F2270
S113245062F31F4200B500BF13009646944610393C
S113246028BFA0E80C50FAD85FEA417C28BF0CC012
S113247048BF40F8042BC90728BF20F8022B48BFE7
S113248000F8012B00BD00F067B9134680B50A4679
S113249001461846FFF7CCF9002002BD70B510F0D4
S11324A0030F0C46154612D0B0F1005F0FD221186D
S11324B0491EB1F1005F0AD3C0F1005632462946E5
S11324C0FFF7B6F9A21B71194FF0005001E0224644
S11324D02946FFF7ADF9002070BD10B514460A4631
S11324E02146BDE810400123FDF7C2BF4FF0FF3184
S11324F00160002141607047F0B585B004460D4687
S11325001646684600F0ACF901208DF80B002068EF
S113251001901B48009000208DF80A00ADF80800D7
S11325207EB1FFF7CBF9174F6946384600F067F9DB
S113253032462946384600F098F938680190FFF78A
S1132540C3F90198206060683018606005B0F0BD80
S113255038B504460D46207910F0030007D06946CB
S113256000220A60C0F104022046FFF7C5FF20687C
S113257028600548016821F48021016031BD000014
S1132580B71DC104002003403C80044070B50D0019
S113259082B00446164601D1002076BD6A4600F09A
S11325A071F830B9009BDB685B68324629462046E7
S11325B0984776BD70B50D0082B00446164601D129
S11325C0002076BD00F07FF800B14CE000F047F841
S11325D068B9009BDB689B683246294620469847C9
S11325E04E49002806BF009AD26800220A6076BDD0
S11325F038B504460D466A4600F044F8A0B9009880
S1132600C068406908B9662032BD2946204600F0FA
S11326105AF810B142F2D87032BD009AD2685269A9
S113262029462046904732BD002DFCD1002032BD02
S113263070B50D0082B00446164601D1002076BD67
S113264000F041F800B10EE000F009F830B9009B49
S1132650DB68DB68324629462046984776BD6A46E1
S1132660294620460EE042F2D87076BD10B52B4CB8
S11326702168002029B109690A0002D08847002195
S1132680216010BD70B542F2D873D2B1244C646895
S1132690146011B915E01034146014688CB1256805
S11326A0002D04BF6668002E01D1E6684EB1A84231
S11326B024BF65688542EED30818401E854228BFB2
S11326C00023184670BD70B50918491E0022144B2A
S11326D09C685D682469160104EBC204583475597A
S11326E066682468AC4208BFAE4205D0864228BF63
S11326F0A14201D3012070BD521C022AE8D300205C
S113270070BD10B50648446804E00068010018BFB5
S113271080471034E0680028F7D110BD0482FF1F01
S11327201080FF1F10B582B000228DF800200A46E9
S1132730064C014604F120002469646C6B46A047F2
S11327409DF8000000B1012016BD00001080FF1F9D
S1132750002200F0B3B800001A480068000B00F033
S11327600F00C01E08282BD8DFE800F005080B0E68
S11327701114172A1A004FF4804013E04FF4C0409C
S113278010E04FF400400DE04FF440400AE04FF4F5
S1132790803007E04FF4C03004E04FF4003001E033
S11327A04FF48020084949680322B0FBF2F0C0F1DD
S11327B0005241F8102F6FF0604202EB4000486075
S11327C000207047007004401080FF1F0B7A4A7A83
S11327D01B0703F0405343EA82728B7A42EA836216
S11327E0CB7A1B0603F080731A4382600B68436044
S11327F042F0007383604968016082607047E0B50D
S1132800164A136843F4802313600A7B002A0A687B
S113281000924A6801920DD14A7A02B102228DF8DF
S113282008200A7A002A14BF022203228DF8092004
S11328308A7A0AE000228DF808200A7A002A14BF56
S1132840022203228DF8092000228DF80A20C97A79
S11328508DF80B106946FFF7B9FF07BD3C800440B3
S11328600FF248011022FEF7F3BF03E011F8013B19
S11328700370521E3AB111F00303F7D103E051F88B
S1132880043B0360121F042AF9D2002A03E011F862
S1132890013B0370521EFAD1704701688068C0F38F
S11328A0017002282CBF080C88B270472110000068
S11328B0FFFF00000000000000000000401810F0BE
S11328C0030308D0C91A1FD3DB0748BF00F8012D42
S11328D028BF20F8022D130030B4144615461039D1
S11328E028BF20E93C00FAD8490728BF20E90C009A
S11328F048BF40F8042D890028BF20F8022D48BFA6
S113290000F8012D30BC7047C91818BF00F8012D1C
S1132910CB0728BF00F8012D7047000001280ED80E
S11329200FF2240280560122012900F01F0102FA4D
S113293001F10CBF024A034A400942F820107047D3
S113294000E100E080E100E01A1B0000BFF34F8FBC
S11329500548064A016801F4E06111430160BFF3D0
S11329604F8F00BFFDE700000CED00E00400FA0506
S1132970ECE7EBE7EAE7E9E701280ED80FF22402D7
S113298080560122012900F01F0102FA01F10CBF57
S1132990024A034A400942F82010704700E100E06F
S11329A080E100E01819000002280ED80FF224027A
S11329B080560122012900F01F0102FA01F10CBF27
S11329C0024A034A400942F82010704700E100E03F
S11329D080E100E01F212300002101807047F0B551
S11329E085B004460D4616466846FFF739FF0020B9
S11329F08DF80B002088019041F221000090002006
S1132A008DF80A00ADF808008EB1FEF757FF0E4F9F
S1132A1069463846FFF7F3FE324629463846FFF743
S1132A2024FF3846FFF739FF0190FEF74DFF019868
S1132A30208005B0F0BD008808800448016821F4B6
S1132A408021016070470000002003403C80044066
S1132A5040684A49405C704748498A6842B14A68BC
S1132A6013780370501C48608868401E8860704763
S1132A700021017070475A2807D1404A01238B5422
S1132A800FF2090111615169084770473B494969CF
S1132A9008477FB5394D696104460FF2F800616853
S1132AA050F82160684600F0E7F801208DF808002E
S1132AB08DF8090002213248E86032482861A26892
S1132AC0606890476946304600F08CF82E493046DD
S1132AD000F004F960680121FFF720FF61684919DB
S1132AE00120887004B0002070BD70B50546234CE9
S1132AF068680119897889B10FF2980151F820604A
S1132B000021FFF70BFF304600F0C2F86868AA689E
S1132B1000219047696809190020887070BD174822
S1132B204160826081680029FCD10020704770B543
S1132B3004460FF2600082B050F82450E86A0001A5
S1132B400BD54FF0006007E0F168684688479DF8B0
S1132B50000068634FF00070E862E86A074E800185
S1132B60F2D4E86A800308D5A86B4FF40031E96217
S1132B7021463269C0B29047F3E773BD7080FF1FEE
S1132B80592A0000772A00000000020A0020CEE73C
S1132B900120CCE700C0024000D00240010C01F14A
S1132BA0804101F58E2101230A6803FA00F01043E5
S1132BB0086070470029016814BF21F4804141F482
S1132BC080410160704700210FF2441252F8213015
S1132BD0834202D0491C0229F8D3084670470121D8
S1132BE02046E7E738B504460D46FFF7ECFF00F052
S1132BF03EF8FFF7F4FF00F083F80122206840005C
S1132C004008206020680840297B40EA8170A97B45
S1132C1040EA8160697B40EA0160E97B00F01CF8CE
S1132C200121204600F04FF8287804EB8000C168A9
S1132C306A6821F0FE41521E41EAC2612A7A920674
S1132C4002F0806211436A7A520602F00072114364
S1132C50C16000F007F831BD090201F44071084376
S1132C6020607047206840084000206070470FF2E1
S1132C70A80151F8200091E700210170082141606A
S1132C80002101724172017341738173C1737047F2
S1132C9010B504460021206800F034F8FFF7A0FFC7
S1132CA000F02CF80FF2700151F82000010C01F132
S1132CB0804101F58E2101230A6803FA00F022EA1B
S1132CC00000086010BD0368090401F47C11012AA6
S1132CD00CBF194323EA0101016070478A0103D53F
S1132CE0026B22F0807202638A0303D5026B22F422
S1132CF080320263026B114301637047204662E72E
S1132D002068024940F0010020607047FFCCFFBA00
S1132D1000C0024000D002400C003C100D003C10EA
S1132D20010C01F1804101F58E2101230A6803FAA7
S1132D3000F0104308607047010C01F1804101F577
S1132D408E2101230A6803FA00F022EA00000860D9
S1132D5070470029817814BF41F0800101F07F01A0
S1132D608170704700210FF2F00252F82130834243
S1132D7002D0491C0229F8D3084670474A0603D5F5
S1132D80827842F040028270890603D5817941F04D
S1132D90200181717047C1788279520648BF41F49D
S1132DA080418079C00648BF41F48051084670478D
S1132DB038B504460D46FFF7D5FF00F030F8A87A81
S1132DC010B1022804D00DE0E8884000207009E02A
S1132DD0E8884000207028894000E071607940F064
S1132DE008006071A078A97800F0FD0040EA410075
S1132DF0297840EAC110A0706079297900F06F0049
S1132E0040EA0110697840EAC110E97800F001F85D
S1132E1031BD00F0DF0040EA4110607170470FF2ED
S1132E20400151F820007BE710B504460021FFF76C
S1132E3090FF2046FFF796FF0FF2240151F820007F
S1132E40BDE8104078E70021817241708170C17043
S1132E500171012101707047006006400070064056
S1132E60060034100700341000210FF2501252F8FB
S1132E702130834202D0491C0329F8D30846704705
S1132E80F8B50D46044628680101B2FBF1F6B6B266
S1132E9006B901265301B3FBF1F1A1EB461751002A
S1132EA0720112FA87F2B1FBF2F1091A6422B0FB43
S1132EB0F2F000EB4000884202D240F2F530F2BD5D
S1132EC02046FFF7D1FF00F043F81043086007F0F5
S1132ED01F01E07800F0F300E070207800F0E000DB
S1132EE040EA262020706670A07A00F0E0000843D3
S1132EF0A072A078297900F0EC000843A0706879EA
S1132F00E074A8796075207C40F088002074607CAF
S1132F1040F0C0006074E078E97909B140F008003D
S1132F20297A09B140F00400E0700020F2BD80B5B8
S1132F30017D0029FCD101794906FCD50021C1702D
S1132F40FFF792FF00F004F822EA0000086001BDD8
S1132F500FF2740151F82000010C01F1804101F5D8
S1132F608E2101230A6803FA00F070474FF4E1311F
S1132F700160002101714171012181710021C17140
S1132F800172704702780A430270C27842EA112241
S1132F90C270827942EA11428271427C42EA116132
S1132FA04174704705E003791B06FCD511F8013B19
S1132FB0C37113465A1E002BF5D1704700A006407A
S1132FC000B0064000C006400A0034100B00341064
S1132FD00C0034100029817814BF41F0800101F005
S1132FE07F018170704700209AE0012098E04068DA
S1132FF06549405C704764498A6842B14A681378FD
S11330000370501C48608868401E88607047002127
S1133010017070475C49496908475A2806D15A4AE1
S113302001238B5459491161516908477047FEB512
S1133030554D044669616068A2680221904766683C
S11330400FF2581050F826706846FFF7FCFE102067
S1133050ADF8060069464E488068006990F879002A
S1133060FF2818BFADF806003846FFF7A1FE01217E
S11330703846FFF7AFFF40213846FFF77FFEFFF7E2
S1133080A9F94FF47A71B0FBF1F04249B1FBF0F0C9
S1133090002100E011464A1C00FB02F3322BF9D355
S11330A021B9B0F5FA7F04D8012102E0202928BF14
S11330B01F21B87900F0F0000843B87101213046AF
S11330C0FFF75AFC34482861012061684919887067
S11330D00020FEBD70B505462B4C6868011989783F
S11330E0A9B10FF2B80151F820600021FFF744FCA8
S11330F000213046FFF76EFF3046FFF795FE686803
S1133100AA6800219047696809190020887070BD79
S11331101D484160826081680029FCD1002070470D
S113312038B505460FF2740050F825402046FFF7E5
S113313032FE00F01201E17000F05001102911D0AC
S11331404106114A14D54007A0780CD540F0100070
S1133150A07000208DF800006846D16888479DF86B
S11331600000207131BD00F0EF00A070207931BD66
S1133170A178C90603D5C007EBD5A078F3E7207979
S113318012692946904731BD8880FF1F1530000021
S11331901080FF1F40420F001B30000000600640FB
S11331A00070064010B598488068006900F1680412
S11331B034214AF2C030FFF7B5FA48B934224AF252
S11331C0C0312046FEF744FB20689049884204D071
S11331D0FF2234212046FFF739F9FFF735F90020A3
S11331E010BD38B5884DA86804694B20E07004F11F
S11331F010020220A0700421002060702070502072
S1133200E0710120A071022060710020207154201F
S1133210E0720120A07200206072207201202063FD
S11332204EF6FF70606305F120002B69DB6A984756
S11332302B69DB6A04F11402012100F060F82B69A8
S1133240DB6A04F11802002100F059F82B69DB6AEB
S113325004F11C02022100F052F82B69DB6A04F12C
S11332602002032100F04BF82B69DB6A04F14402CD
S1133270052100F044F82B69DB6A04F148020621B9
S113328000F03DF82B69DB6A04F14C02072100F0E1
S113329036F8A0695E4A404252424FF0FF31024084
S11332A0891A5C4AE1651040A06500215A482066ED
S11332B05A4860666869E16007E094F87830134220
S11332C002D0E3681A43E260491C182202FB01029F
S11332D01268002AF1D15248016821644168E1630F
S11332E08068A063686850F8101F616241680068D4
S11332F0081A401CA06201202065002032BD05F19F
S113330020001847F8B514463F4A464F91680426F2
S1133310401E096917281D464BD8DFE800F00C123F
S11333201416181A204A4A22242B4A1C1E2E313DF8
S1133330404244464A4805B12E6004B12160002051
S1133340F2BD0C31F7E71031F5E71431F3E718312A
S1133350F1E72031EFE72431EDE72831EBE73431B1
S1133360E9E73031E7E7D06941694969884738605E
S11333703946E0E710265831DDE72B480068F6E7C8
S113338002F1200012699269694690479DF8000095
S11333900028ECD00120EAE70C263831CBE7443191
S11333A0C9E74831C7E74C31C5E75031C3E70831B5
S11333B0C1E742F63C00F2BD134A92681369401E0D
S11333C0062842F63E0218D909380AD0401E0128C0
S11333D084BFC01E032810D9083808D0801E0CD022
S11333E00EE0002918BF012903D11963704703298E
S11333F001D3104670471965704742F63D00704787
S113340042F63C00704700001080FF1F6B63666744
S1133410DC3A0000000000000080FF1FF785FF1F5A
S113342058800440CC82FF1F2480044030B50446F9
S113343085B060686946FDF783F9002835D1606876
S1133440012804D002280CBF424D434D00E0434DF7
S113345001A8FFF78BFD0098019001208DF80B0067
S11334608DF80C006068FEF7C3FF024601A92846E8
S1133470FFF706FDB0B960680121FFF795FA4FF434
S113348000512846FFF77EFD6068A268344C022193
S1133490904761685A2088476168A62088470120C0
S11334A0207003E06068FDF731F9002005B030BDFD
S11334B010B504462A4841606068A268012190471B
S11334C06068FDF723F9002010BD10B504462448B8
S11334D0007870B160680021FFF766FA606801281F
S11334E004D002280CBF1B481B4800E01B48FFF710
S11334F01EFD6068FDF722F96068A268BDE810400F
S11335000021104780B54068012804D002280CBF70
S11335101048114800E01148FFF744FD002002BDA7
S113352010480178890600D50AE070470E480178F2
S11335308A0701D5C0787047890600D500E0704736
S1133540C07807494968084708480178890600D5C2
S1133550F6E7704700C0064000A0064000B00640F1
S11335605883FF1F04A0064004B0064004C0064070
S1133570AF49D1F88820531C5218C1F8883082F81A
S11335802000D1F8880000F03F00C1F8880070479F
S113359000207047B8E02DE9FC410C00154614BF2B
S11335A0002D0420984628D0A14F002007F1900652
S11335B02860707000F0A8F818B11EE0A22000F096
S11335C075F820213846FDF78DFD42463946684698
S11335D000F0F8F810B1002129600EE03946684681
S11335E000F042F9BDF804108142E7D101203070A7
S11335F02760BDF8020028600020BDE8F6812DE9AF
S1133600F0410C0082B015461E4635D0212D33D230
S113361000F07AF800283FD1DFF8148298F891007E
S113362010B1002088F8910008F160075A20387022
S1133630A42078700EB1A52078707D802DB12A4623
S1133640214608F16600FEF7F3F808F166013846F2
S113365000F00AF9B880A91D384600F064F8D8B91A
S1133660684600F0EFF8B8B99DF80100A12812D01F
S1133670A22806D0A32801D004200DE042F2127043
S11336800AE07888811D384600F04DF820B99DF88D
S11336900100A228E4D00020BDE8F681654801219C
S11336A081700021017070472020704780B55A2135
S11336B08DF800108DF8010001205D4981F891001A
S11336C00221684600F02FF802BD10B5044659489F
S11336D082B00178427880781140014211D10FF212
S11336E0B8100088ADF80000022223695B686946BF
S11336F02046984723690FF2A4115B6808222046EC
S1133700984742F2137016BD4A48017819B1002156
S11337100170A12004E0817819B100218170A320F7
S1133720C4E700207047444AD3690A460146184654
S11337301B695B6818472DE9F14F8B461646FDF768
S113374084F804464FF47A7088467043FDF78DF888
S1133750DFF8DCA00027064689460AF188050EE05A
S11337606868296888420CD05044009990F8200079
S113377078547F1C6868401C00F03F0068605F4517
S11337801DD0FDF762F8021B61EB080341450AD81E
S113379028BFA04207D2E2436FEA08031018594138
S11337A0421C41F10003B9F1000F08BF002ED7D02D
S11337B04B45D5D301D8B242D2D3052000E0002036
S11337C0BDE8F28F70B582B005460C46164600F08F
S11337D039F858BB6878A62804D11748C069FFF7A0
S11337E074FF76BDA42106B1A521884201D0012031
S11337F076BD00F023F8BDF800106980B0B9084622
S11338002128A8BF2020688000F018F8BDF8001017
S1133810A98058B9698849B12046FEF799FF69889B
S11338200A2000FB01F22046FFF785FF76BD000069
S11338306083FF1FF083FF1F1080FF1F14220221EB
S1133840684678E710B50446002201212046FFF7B8
S113385072FF40B920785A28F6D1601CBDE81040A8
S11338600A22012167E710BD30B583B004460D4636
S11338706846FFF7B1F8042221466846FFF7AFF81F
S1133880628829466846FFF7AAF801A96846FFF747
S1133890D2F8BDF804003EBD5AA700000002015052
S11338A00000AAEA05484CF22051C1814DF62811C6
S11338B0C1814FF4E9710180704700BF00200540C9
S11338C000F00BF8002801D000F00AF80020C046F0
S11338D0C046FEF7F9F8FEF713F90120704700001F
S11338E010B5074979441831064C7C44163404E079
S11338F00A68081D511888470146A142F8D110BD35
S1133900CC010000D80100003D0A00004B0A000071
S1133910EC0400003081FF1F34060000A080FF1F6C
S1133920C40600000080FF1F7C0500006406000040
S11339300000000000000000000000000000000083
S11339400000000000000000000000000000000073
S11339500000000000000000000000000000000063
S11339600000000000000000000000000000000053
S11339706881FF1FA881FF1F0000000000000000F5
S113398000000000592A0000772A0000000000000F
S1133990000000000000000000000000F72F0000FD
S11339A01B3000000000000000000000FFFF0700C3
S11339B001000000040600000080FF1FFFFF00203C
S11339C0010000004C06000000000040FFFF07401B
S11339D000000000D405000000F00F40FFFF0F407E
S11339E000000000D4050000000000E0FFFF0FE02D
S11339F000000000D40500000000000000000000EA
S1133A0000000000000000000000400130B504E0A8
S1133A1012F8014B00F8014B491ED1B1C507F7D488
S1133A200129F5D0850701D4042904D232F8024BC8
S1133A3020F8024B891E8B08EFD000EB830403E0CF
S1133A4052F8045B40F8045BA042F9D3A1EB830174
S1133A50E3E730BD80B513460246184600E080B562
S1133A60FFF7D4FF002002BD10B514460A462146D4
S1133A70BDE810400123FCF7FBBCFFF7FEBFC046C6
S1133A80C046C046C046FFF71BFF19E050F8041BB0
S1133A90CB0744BFA9F101035918121F0023042ABC
S1133AA041F8043BF9D25FEA827C0B4604D54FF01F
S1133AB0000CA1F800C09B1CD10744BF0021197061
S1133AC050F8042B002AE1D170470000BFFFFFFF2C
S10F3AD0EC0200000881FF1F0000000051
S9030411E7
